:100000003BC0A6C154C053C052C051C050C04FC025
:100010004EC04DC04CC04BC04AC049C048C047C08C
:1000200046C045C044C0040309041C0377007700A0
:1000300077002E00660069007300630068006C00A2
:100040002E00640065000E0355005300420061005D
:100050007300700012011001FF000008C016DC05DB
:1000600003010102000109021200010100801909C7
:10007000040000000000000011241FBECFE5D4E002
:10008000DEBFCDBF10E0A0E6B0E0EAE6FFE002C0D0
:1000900005900D92A436B107D9F710E0A4E6B0E0C0
:1000A00001C01D92A93AB107E1F7DBD45CC7A8CF24
:1000B00085B7836085BF8BB780648BBF08951F931E
:1000C000CF93DF9360918900635067FD13C08091E7
:1000D0008600CCE0D0E0C81BD109C357DF4F809128
:1000E00085008D3209F462C08091640087FD84C070
:1000F000109289008091600084FF4AC06091610085
:100100006F3F09F445C0693070F168506093610039
:100110008091790098E889278093790068E0809140
:10012000640087FD8BC0209187003091880086FF96
:100130006DC0AAE7B0E080E090E0F901E80FF91F98
:10014000E491ED9301966817C1F76150862F90E016
:100150006F5F0196820F931F9093880080938700B2
:10016000162F1C5F0BC0109261008091790098E8F7
:10017000892780937900662391F614E08AE790E05E
:10018000E3D01C3019F08FEF809361001093600072
:1001900094E186B3837031F49150D9F710928A00BC
:1001A00010928400DF91CF911F910895683009F07B
:1001B0009FCF83EC809379008AE580936000109252
:1001C00064008881807659F59A8110928200898135
:1001D000882309F043C01092830022E082E890E077
:1001E00090938800809387008F81882319F49E81E3
:1001F000921708F1922F1FC0CE0144D48F3F51F1C6
:10020000882309F475CF1092610072CF962FD9011F
:10021000EAE7F0E08D9181939150E1F796CFCE011E
:1002200023D5282F8F3F01F7888187FD25C09FEFB9
:1002300080E880936400909361005ACF8AE790E051
:10024000C3D4682F893008F453C08FEF80936100C6
:100250001EE19CCF8EE1809360004ACF853071F023
:10026000863091F0883031F1893061F18A3031F196
:1002700020E082E890E0B4CF9E81DACF90938A00AC
:1002800020E082E890E0ACCF8B81813049F1823070
:10029000F9F0833029F020E080E480936400A4CF5B
:1002A000992349F586E290E0909388008093870037
:1002B00024E0F2CF21E08CE890E092CF21E082E8C8
:1002C00090E08ECF90938C0020E082E890E088CF81
:1002D00086E690E0909388008093870022E1DCCF4F
:1002E00084E590E0909388008093870022E1D4CF4A
:1002F000182F1C5F43CF913051F0923061F686E4A5
:1003000090E090938800809387002EE0C5CF8AE22A
:1003100090E090938800809387002CE1BDCFA82FB8
:10032000B92F80E090E041E050EA60956F5F58F4AB
:100330002D9138EF82279795879510F08427952780
:100340003F5FC8F3F3CF0895EADF8D939D9308953F
:10035000CF93CFB7CF93C395B09BE9F7B09B09C0BC
:10036000B09B07C0B09B05C0B09B03C0B09B01C051
:10037000A1C0DF93C0918600DD27C357DF4FB09B3C
:1003800002C0DF91EBCF2F930F931F9306B32FEF94
:1003900000FB20F94F933F9316B34FEF012700FB6B
:1003A00021F93BE031C04E7F012F16B3216028C0F8
:1003B000102F4D7F2260000006B329C04B7F2460C0
:1003C000012F000016B32BC016B3477F28602AC048
:1003D0004F7E06B320612CC04F7D16B320622FC024
:1003E0004F7B06B3206432C0422706B349934FEFD8
:1003F0000000102710FB20F916B31370C9F1297FF4
:1004000091F2012700FB21F906B3237F89F23150D5
:1004100058F1102710FB22F916B3277E79F2012735
:1004200000FB23F92F7C81F206B3102710FB24F97F
:100430002F7971F200C016B3012700FB25F92F7345
:1004400059F200C006B3102710FB26F9223040F203
:1004500000C016B3012700FB27F9243028F64F7798
:10046000206816B30000F9CF10E41ABF002717C0A8
:100470003B503195C31BD04010E41ABF0881033CA8
:10048000E9F00B34D9F0209184001981110F121377
:10049000EDCF093641F10D3211F0013E39F70093ED
:1004A0008B003F914F911F910F912F91DF91CAB710
:1004B000C6FD51CFCF91CFBFCF91189520918B0022
:1004C000222379F310918900112311F5343012F1B0
:1004D0003093890020938500109186003BE0311B0A
:1004E0003093860017C00091890001308CF40AE532
:1004F0003091600034FD10C000936000C9E7D0E087
:100500000FC02795A8F45150A9F4220F0000F9CF8D
:100510004AE503C042ED01C0432FC4E1D0E032E020
:1005200017B31360C09A17BB08B320E413E05F93BE
:10053000012756E008BB279520F4515021F4220FE3
:10054000F9CF012756E000003B5A08BBD0F22795AF
:1005500028F4515029F4220F0000F9CF012756E06A
:10056000279508BB20F4515021F4220FF9CF012721
:1005700056E02991332308BB21F60C7F10918A00A5
:10058000110FC651D04008BB11F01093840010E445
:100590001ABF016017B31C7F402F4C7F5F9100C0D2
:1005A00000C008BB17BB48BB7CCF8091A6008DB9AB
:1005B0008091A3008EB90895282F8830B8F080E983
:1005C00093E09093A5008093A4001092A30029309B
:1005D00089F12A30E0F02B30C9F12C30D1F481E5DB
:1005E0008093A60081E08093A30008958FE693E0B6
:1005F0009093A5008093A400243001F1253080F071
:100600002630C1F1263090F12730E1F008952830EE
:1006100009F182E58093A60081E08093A30008950C
:10062000223001F12330D0F4213081F780EC809327
:10063000A700089582E58093A600089588E180933D
:10064000A700089583E08093A700089581E5809333
:10065000A600089583E58093A600089580E3809323
:10066000A700089580E68093A70008958CE080930A
:10067000A70008952093A700089522B79091A7009E
:1006800082B7821B8917E0F3089587B38C6287BB1A
:10069000C298C59892B72091A70082B7891B82178C
:1006A000E0F3C29A92B782B7891B8217E0F3C2982F
:1006B0008091A4009091A5008059934009F008957D
:1006C0008091A6008DB98091A3008EB9089587B35B
:1006D000837D87BB88B3837D88BB1DB80895582F61
:1006E0002091A70040E030E057FD16C0C398440FAA
:1006F000B4994F5FC59A92B782B7891B8217E0F30E
:10070000C59892B782B7891B8217E0F33F5F3830F4
:1007100029F0550F57FFEACFC39AE9CF842F0895E8
:100720008FB9779BFECF8FB108950F931F930FE181
:10073000E091A400F091A5008CEA0995E091A40055
:10074000F091A50083E50995E091A400F091A50042
:1007500080E00995182FE091A400F091A50080E0B9
:100760000995133509F444C01DB8C59A92B7209174
:10077000A70082B7891B8217E0F3C59892B782B7AA
:10078000891B8217E0F3002371F0902F9150E091C4
:10079000A400F091A50083E0E039F807A9F0002358
:1007A000D9F0092FC9CF90916200923020F080914A
:1007B000A8008823A9F09FEFE091A400F091A50084
:1007C00083E0E039F80759F78091A6008DB9809150
:1007D000A3008EB9002329F781E01F910F9108959E
:1007E000892F815080936200E7DE08E097E0CFCF49
:1007F00080E01F910F910895EF92FF920F931F9346
:100800007B018C01862F8170880F880F880FE09103
:10081000A400F091A50080620995D801C70129E0E4
:10082000B695A795979587952A95D1F7E091A4005D
:10083000F091A500099516950795F794E794E09136
:10084000A400F091A5008E2D0995E091A400F091EF
:10085000A50080E009951F910F91FF90EF900895FA
:100860000F931F938C01E091A400F091A50080EA02
:100870000995E091A400F091A500812F0995E091E0
:10088000A400F091A500802F0995E091A400F091BB
:10089000A50080E009951F910F910895FF920F9395
:1008A0001F938C01F62EE091A400F091A50080EC3E
:1008B0000995E091A400F091A500812F0995E091A0
:1008C000A400F091A500802F0995E091A400F0917B
:1008D000A5008F2D09958EE1B7D080E01F910F9173
:1008E000FF900895CF92DF92EF92FF920F931F93A4
:1008F0006B017C01142FE091A400F091A5008CE421
:100900000995D701C60149E0B695A79597958795B2
:100910004A95D1F7E091A400F091A5000995D7017F
:10092000C601B695A79597958795E091A400F0919B
:10093000A5000995E091A400F091A50080E009953B
:100940001F3FF1F012B70EE1C701B60155DF8F3F2F
:1009500079F482B7811B8D33B8F312B70150A1F738
:1009600081E01F910F91FF90EF90DF90CF9008955D
:1009700080E01F910F91FF90EF90DF90CF9008954E
:100980008FE062D080E01F910F91FF90EF90DF9099
:10099000CF900895CF92DF92EF92FF920F931F9323
:1009A0006B017C01042F122F862F8170880F880F16
:1009B000880FE091A400F091A50080640995D7010B
:1009C000C60169E0B695A795979587956A95D1F781
:1009D000E091A400F091A5000995D701C601B69554
:1009E000A79597958795E091A400F091A5000995AA
:1009F000E091A400F091A500802F09951123C1F08A
:100A00000F37F1F012B70EE1C701B601F5DE8F37EF
:100A100079F482B7811B8D33B8F312B70150A1F777
:100A200081E01F910F91FF90EF90DF90CF9008959C
:100A300080E01F910F91FF90EF90DF90CF9008958D
:100A40008FE002D080E0F5CF382F882349F020E0F6
:100A500092B782B7891B8C33E0F32F5F2317C0F363
:100A6000089512BA18BA8BEF81BB8FEF87BB17BA04
:100A700093E094BB8EEF85BB93BF1ADB78941FDBAA
:100A80001EDBFDCFFF920F931F93CF93DF93F82EC2
:100A9000292F062F40916500413051F0443041F03C
:100AA0001FEF812FDF91CF911F910F91FF9008953C
:100AB000002309F487C08F2D922F9C01E90110E0DB
:100AC00053C08091750090917600892B09F058C031
:100AD0006091710070917200809173009091740028
:100AE000488121E057DF809166009091670001976F
:100AF0009093670080936600892BD9F4109265006B
:100B00008091770081FF3AC08091780090E0209139
:100B10007500309176008217930781F16091710022
:100B20007091720080917300909174004881DADEB8
:100B300011E08091710090917200A0917300B091CA
:100B400074000196A11DB11D8093710090937200F5
:100B5000A0937300B093740021969E012F19201763
:100B600008F09FCF40916500413009F4AACF8091F1
:100B7000710090917200688191DEB5CF11E0D9CFFC
:100B80006091710070917200809173009091740077
:100B9000488120E0FFDE80917800815080937800CA
:100BA000882309F0A0CF609171007091720080914C
:100BB000730090917400488195DE80917500809358
:100BC000780091CF10E06DCF0F931F93CF93DF93F9
:100BD000082F162F40916500842F8250823038F004
:100BE0001FEF812FDF91CF911F910F910895662301
:100BF00099F1802F9C01E90120C0809171009091B2
:100C000072002EDE88838091710090917200A09115
:100C10007300B09174000196A11DB11D8093710005
:100C200090937200A0937300B093740021969E017C
:100C3000201B211778F4409165004230F1F6609155
:100C40007100709172008091730090917400D4DDF6
:100C50008883D9CF183028F610926500812FDF9154
:100C6000CF911F910F9108950F931F93CF93DF930F
:100C70008C01DC0111969C91913009F447C09230AF
:100C800009F4E4C0933009F45DC0943009F4B2C0B3
:100C9000973009F483C0953009F44AC1963009F4BD
:100CA000E6C0983009F02AC1809168008823B1F429
:100CB000D80113969C91139780E012962C9130E006
:100CC000822B932BAA2797FDA095BA2F80937100B2
:100CD00090937200A0937300B0937400109276000A
:100CE0001092750010927700F801978180E02681BC
:100CF00030E0822B932B909367008093660084E012
:100D0000809365008FEFC9E6D0E013C01092A80071
:100D10009A9905C085E0809362009093A800809125
:100D200062004ADC10926800A998AFDC80E0C9E656
:100D3000D0E0D0938800C0938700DF91CF911F91BE
:100D40000F910895E091A400F091A500D8011296AA
:100D50008C910995C9E6D0E080936900E091A400E8
:100D6000F091A500D80113968C91099580936A00A3
:100D7000E091A400F091A500D80114968C910995FA
:100D800080936B00E091A400F091A500D801159626
:100D90008C91099580936C0084E0CBCF80916800A2
:100DA000882399F4F801938180E0228130E0822B3E
:100DB000932BAA2797FDA095BA2F8093710090934B
:100DC0007200A0937300B0937400D80117969C91A1
:100DD000179780E016962C9130E0822B932B9093FE
:100DE00067008093660083E0809365008FEFC9E61B
:100DF000D0E09FCF80916800882399F4F801938117
:100E000080E0228130E0822B932BAA2797FDA095CA
:100E1000BA2F8093710090937200A0937300B093E7
:100E20007400D80117969C91179780E016962C9124
:100E300030E0822B932B909367008093660082E0D2
:100E4000809365008FEFC9E6D0E073CF40DCA99AAC
:100E50008091A800882339F48CE08093620080E0C0
:100E6000C9E6D0E066CF80E0C9E6D0E062CF8091ED
:100E70006800882399F4F801938180E0228130E0B2
:100E8000822B932BAA2797FDA095BA2F80937100F0
:100E900090937200A0937300B0937400D8011496DD
:100EA0008C91149715969C91292F2F702093770081
:100EB000492F50E0407F507042955295507F542703
:100EC000407F5427480F511D509376004093750082
:100ED00020FF02C040937800F801978180E02681CE
:100EE00030E0822B932B909367008093660081E023
:100EF000809365008FEFC9E6D0E01BCF9930F9F001
:100F00009A3009F0B0CFD80112969C91809162007E
:100F1000981740F4992331F08091A800882311F4A8
:100F200090936200C9E6D0E01092690081E001CFA1
:100F3000FCDBC9E6D0E08093690081E0FACE81E075
:100F400080936800F80182819381A481B5818093A8
:100F5000710090937200A0937300B093740080E0CE
:0A0F6000C9E6D0E0E6CEF894FFCF1A
:040F6A005AFF0C001E
:00000001FF
